:0200000480007A
:100000006F00C0006F20C02B6F20802B930000007A
:10001000130100009301000013020000930200008E
:100020001303000093030000130400009304000076
:10003000130500009305000013060000930600005E
:100040001307000093070000130800009308000046
:100050001309000093090000130A0000930A00002E
:10006000130B0000930B0000130C0000930C000016
:10007000130D0000930D0000130E0000930E0000FE
:10008000130F0000930F00009702000093820201FB
:10009000739052307350447497020000938202F7B9
:1000A0007390523017D100001301C1E3F32240F1E5
:1000B0009392C2003301510073100134EF20D0132A
:1000C000173500001305C5946F20407383328510E7
:1000D000739012148330850003310501833185014B
:1000E000033205028332850203330503833385031C
:1000F00003340504833485048335850503360506FA
:1001000083368506033705078337850703380508D7
:10011000833885080339050983398509033A050AB7
:10012000833A850A033B050B833B850B033C050C97
:10013000833C850C033D050D833D850D033E050E77
:10014000833E850E033F050F833F850F033505056D
:10015000730020107311011423341100233C31006B
:10016000233041022334510223386102233C7102BF
:1001700023308104233491042338A104233CB104A7
:100180002330C1062334D1062338E106233CF1068F
:10019000233001092334110923382109233C310973
:1001A0002330410B2334510B2338610B233C710B5B
:1001B0002330810D2334910D2338A10D233CB10D43
:1001C0002330C10F2334D10F2338E10F233CF10F2B
:1001D000F312011423385100F32200102330511080
:1001E000F322101423345110F32230142338511009
:1001F000F3222014233C5110130501006F20C03757
:1010000000000000000000000000000000000000E0
:1010100000000000000000000000000000000000D0
:1010200000000000000000000000000000000000C0
:1010300000000000000000000000000000000000B0
:081040000000000000000000A8
:10200000B367B500B3E7C70093F77700B306C50021
:10201000638407023386C50093070500637ED502FB
:1020200003C705009385150093871700A38FE7FE6C
:10203000E398C5FE67800000E37ED5FE93070500A8
:1020400003B70500938787009385850023BCE7FECF
:10205000E3E8D7FE6780000067800000130101FFFE
:10206000B367C500233081002334110093F7770054
:10207000130405003307C500638207026376E50099
:1020800093F5F50FEFF09FFD8330810013050400F9
:1020900003340100130101016780000093F5F50F7F
:1020A0009717000083B707EEB385F502E37EE5FCE2
:1020B000930705009387870023BCB7FEE3ECE7FE98
:1020C0008330810013050400033401001301010172
:1020D0006780000083470500638E070093070500B3
:1020E00003C7170093871700E31C07FE3385A7403B
:1020F000678000001305000067800000834705002B
:10210000938515001305150003C7F5FF638A0700C3
:10211000E386E7FE1B8507003B05E540678000007E
:10212000130500006FF05FFFB367B50093F777000A
:10213000639E0702137886FF330805016378050361
:10214000930705006F000001938787009385850042
:1021500063F8070183B6070003B70500E386E6FED0
:102160003385A7403306A640138507003386C50094
:102170006F00400103C705008347F5FF93851500F5
:10218000639AE70013051500E396C5FE13050000EA
:10219000678000003B85E7406780000093070500EB
:1021A00003C705009387170093851500A38FE7FEEB
:1021B000E31807FE6780000003470500930600024E
:1021C000930705006318D70003C71700938717000C
:1021D000E30CD7FE9306D0026300D7069306B00245
:1021E0006300D70483C607009305000063820604DA
:1021F0001305000093871700131725001B8606FDA3
:1022000083C607003307A700131717003305E6003E
:10221000E39206FE638005023305A040678000005C
:1022200083C617009305000093871700E39206FC0E
:10223000130500006780000083C617009305100097
:1022400093871700E39606FA130500006FF09FFED0
:1022500083470500638007049305101017F7FFFFFD
:10226000130747DA93950503033607001305150096
:10227000B3E6B700630A060097F7FFFF23B407DC55
:1022800083370700E39A07FE2330D7008347050012
:10229000E39C07FC6780000017F7FFFF130787D652
:1022A00083370700638A070097F7FFFF23BC07D82F
:1022B00083370700E39A07FE2330A7006F00000072
:1022C000130101FF1305903423341100EFF0DFFCFC
:1022D000130101FE1306810093077101130890009A
:1022E0006F008000930707009376F50013870600C0
:1022F000930500036374D800930570053B07B7008E
:102300002380E700135545001387F7FFE31CF6FC15
:1023100083478100230C010063820704130510101A
:102320009306060017F7FFFF1307C7CD1315050324
:10233000833507009386160033E6A700638A0500FD
:1023400097F7FFFF23B007D083370700E39A07FE14
:1023500083C706002330C700E39C07FC130101027A
:1023600067800000130101FB9307100037F7FFFFA0
:102370002322F1002334110423308104233C9102F1
:10238000233821032334310323304103233C5101FB
:1023900023340100B306E500B7E7030063F6F6183F
:1023A0009359C5009384096017390000130989C542
:1023B00093973400B307F90083B707003374E5003F
:1023C0006396071017770000130747C4033A070006
:1023D00063000A1883378A009776000083B686C2A6
:1023E0002330F700638CD712130641009305810058
:1023F00013050400833A0A00EF00C0606310051063
:1024000093D6CA009396A60093E6F60193973400FC
:10241000B307F90013E7060C23B0E70073000412BA
:1024200097270000938707BE93994900B387370128
:1024300003B707006318071203370A00B705040043
:1024400023B0E70003378A0023B4E700F3A50510A3
:10245000B707E0FFB307F4003716000013070400C6
:102460003386C70003B3070083B8870003B80701AA
:1024700003B5870123306700233417012338070190
:10248000233CA7009387070213070702E39CC7FCBE
:102490007390051093973400B304F90023B0D4006F
:1024A000730004120F100000833081040334010410
:1024B000833481030339010383398102033A010222
:1024C000833A8101130101056780000013F70704B7
:1024D0006302070413F70708631207061307F000E7
:1024E00093E70708639CE50493943400B3049900D0
:1024F00023B0F400730004126FF01FFB83360A0050
:102500008337810093D6C6009396A600B3E6F60003
:102510006FF0DFEF93E707046FF01FFD9777000080
:1025200023B207AE6FF05FEC17150000130505A688
:10253000EFF01FD213053000EFF01FD61715000083
:10254000130545A9EFF0DFD013053000EFF0DFD41D
:1025500017150000130585ACEFF09FCF1305300071
:10256000EFF09FD3171500001305C5ACEFF05FCE59
:1025700013053000EFF05FD2130101F82338810614
:10258000233C11062334910623302107233C3105D7
:10259000233841052334510523306105233C710361
:1025A00023388103233491032330A103233CB10159
:1025B00013040500EF0080446312050E8335841177
:1025C000930780006380F510930720006380F50671
:1025D000938745FF130710006376F7009307F00019
:1025E000639CF51E03350411EFF0DFD713050400DB
:1025F00003340107833081078334810603390106E0
:1026000083398105033A0105833A8104033B0104C0
:10261000833B8103033C0103833C8102033D0102B0
:10262000833D8101130101086FD05FAA0337841035
:1026300093773700639E0706EF0780007310300022
:102640000327070083A707006300F7061305101090
:1026500093071004971600009386C6A117F7FFFF93
:102660001307479A13150503833507009386160051
:1026700033E6A700638A050097F7FFFF23B4079CA2
:1026800083370700E39A07FE83C706002330C7009D
:10269000E39C07FC13053000EFF01FC01305040096
:1026A000EFD0DFA26FF09FF113051000EFF0DFBE57
:1026B00017150000130505A6EFF09FB913053000AC
:1026C000EFF09FBD83270405B7140000972A000090
:1026D000938A4A932334F100173D0000130D8D9225
:1026E000B70C0400370CE0FF177A0000130A8A9138
:1026F000977B0000938B8B9137FB030093D7C4002B
:102700001399470033872A0103370700630C070832
:102710009387076093973700B307FD0083B90700DD
:1027200093F709046380070AF3AD0C103384840126
:10273000371600009305040013850400EFF0DF9EB8
:102740006304050493F909086380090AB7160000B9
:102750001387040093070400B386D40003380700EE
:1027600003358700833507010336870123B007014E
:1027700023B4A70023B8B70023BCC7001307070280
:1027800093870702E31CD7FCB3872A0173900D10CF
:1027900003370A0023B00700630007022334F70061
:1027A0002330FA00B7170000B384F400E39864F50F
:1027B00003358100EFF05FAE2330FA0023B0FB0059
:1027C0006FF05FFE171500001305C58DEFF05FA8D1
:1027D00013053000EFF05FAC1715000013050596E8
:1027E000EFF01FA76FF01FEB171500001305058F03
:1027F000EFF01FA613053000EFF01FAAF32740F1FA
:10280000639A0718974700009387C77F130101ED6C
:1028100093D7C70023308112175800001308887E11
:10282000130405009397A700173500001305857D55
:10283000233411129356C5001357C80093E71700AD
:10284000972800009388087C1306F0FF233CF5FED0
:102850009396A6001317A700B707002093E616006B
:102860001367170093D5C8001313F6039387F70C6B
:10287000233CF8FE23B0D8002330E500B3E7650021
:102880007390071873270018639EE7141356B60059
:102890009307F0019702000093824201F3925230B5
:1028A0007310063B7390073A739052301308F0BFD1
:1028B0001318580197E7FFFF9387078AB38707012B
:1028C00073905710F3270034B387070173900714F0
:1028D000B7B700009B87071073902730B7E7010058
:1028E0009B870760739007307350403017270000B4
:1028F000130747B09307083EB3060701B307F70075
:10290000B7080800176600002332D67017230000AE
:10291000130343ED9766000023B6F66E9388F80321
:10292000930720011308080113D61700B386170177
:10293000B347F600B30507019396C6009397570077
:102940002330D7002334B70093F70702130707019A
:10295000B367F600E31AE3FC1306001293050000C8
:10296000130501009727000023BA07E6EFF00FEFE9
:10297000B70700803304F4001305010023348110ED
:10298000EFD0CFF48330811203340112130101130D
:102990006780000013071000B787170A3706080082
:1029A0009387674B1306C6FF1315F7019316E703CA
:1029B0006F00C0012F20070013D71700B3C7E7002F
:1029C0009397E703B3F7D700B3E7E70033F7C70000
:1029D00093F517003307A700E39E05FC03200700CB
:1029E0006FF09FFD1705000013054578EFF05F8637
:1029F00013053000EFF05F8A6780000013050000C8
:102A0000678000001305000067800000930120002C
:102A1000B70001009B8010F093900001938000F0BC
:102A200037110F0F1B01F1F033F72000B713000F20
:102A30009B8303F06318775293013000B710F00FB7
:102A40009B8000FF37110F001B01F1F01311C10033
:102A50001301010F33F72000B703F0009B83030F2E
:102A60006312775093014000B700FF009B80F00F86
:102A700037110F0F1B01F1F033F72000B7030F00E0
:102A80009B83F3006310774E93015000B7000F0053
:102A90009B80F00F9390C0009380F00037110F00DF
:102AA0001B01F1F01311C1001301010F33F72000D6
:102AB000B7030F009B83F3009393C3006314774A1B
:102AC00093016000B70001009B8010F0939000011B
:102AD000938000F037110F0F1B01F1F0B3F02000CD
:102AE000B713000F9B8303F0639E70469301700041
:102AF000B710F00F9B8000FF37110F001B01F1F0A2
:102B00001311C1001301010F33F12000B703F000CE
:102B10009B83030F6318714493018000B700010089
:102B20009B8010F093900001938000F0B3F01000B0
:102B3000B70301009B8313F093930301938303F086
:102B4000639270429301900013020000B7000100ED
:102B50009B8010F093900001938000F037110F0FCD
:102B60001B01F1F033F720001303070013021200DA
:102B700093022000E31C52FCB713000F9B8303F069
:102B80006312733E9301A00013020000B710F00F10
:102B90009B8000FF37110F001B01F1F01311C100E2
:102BA0001301010F33F72000130000001303070087
:102BB0001302120093022000E31A52FCB703F00044
:102BC0009B83030F6310733A9301B000130200005C
:102BD000B700FF009B80F00F37110F0F1B01F1F0C2
:102BE00033F7200013000000130000001303070058
:102BF0001302120093022000E31C52FCB7030F00E3
:102C00009B83F300631073369301C000130200002E
:102C1000B70001009B8010F093900001938000F0BA
:102C200037110F0F1B01F1F033F7200013021200D0
:102C300093022000E31E52FCB713000F9B8303F0A6
:102C4000631277329301D00013020000B710F00F27
:102C50009B8000FF37110F001B01F1F01311C10021
:102C60001301010F1300000033F7200013021200BC
:102C700093022000E31C52FCB703F0009B83030F78
:102C80006312772E9301E00013020000B700FF00EB
:102C90009B80F00F37110F0F1B01F1F013000000A4
:102CA0001300000033F720001302120093022000EB
:102CB000E31E52FCB7030F009B83F3006314772AD3
:102CC0009301F00013020000B70001009B8010F098
:102CD00093900001938000F01300000037110F0F54
:102CE0001B01F1F033F720001302120093022000C1
:102CF000E31C52FCB713000F9B8303F06314772689
:102D00009301000113020000B710F00F9B8000FF39
:102D10001300000037110F001B01F1F01311C10067
:102D20001301010F1300000033F7200013021200FB
:102D300093022000E31A52FCB703F0009B83030FB9
:102D4000631277229301100113020000B700FF0005
:102D50009B80F00F130000001300000037110F0FCD
:102D60001B01F1F033F72000130212009302200040
:102D7000E31E52FCB7030F009B83F3006314771E1E
:102D8000930120011302000037110F0F1B01F1F016
:102D9000B70001009B8010F093900001938000F039
:102DA00033F720001302120093022000E31E52FCAE
:102DB000B713000F9B8303F06316771A930130015A
:102DC0001302000037110F001B01F1F01311C100B5
:102DD0001301010FB710F00F9B8000FF13000000DC
:102DE00033F720001302120093022000E31C52FC70
:102DF000B703F0009B83030F63167716930140011E
:102E00001302000037110F0F1B01F1F0B700FF0094
:102E10009B80F00F130000001300000033F7200028
:102E20001302120093022000E31E52FCB7030F00AE
:102E30009B83F30063187712930150011302000083
:102E400037110F0F1B01F1F013000000B700010054
:102E50009B8010F093900001938000F033F72000E6
:102E60001302120093022000E31C52FCB713000F60
:102E70009B8303F06318770E930160011302000037
:102E800037110F001B01F1F01311C1001301010FE5
:102E900013000000B710F00F9B8000FF130000002C
:102EA00033F720001302120093022000E31A52FCB1
:102EB000B703F0009B83030F6316770A9301700139
:102EC0001302000037110F0F1B01F1F01300000077
:102ED00013000000B700FF009B80F00F33F72000C5
:102EE0001302120093022000E31E52FCB7030F00EE
:102EF0009B83F3006318770693018001B7000100FC
:102F00009B8010F093900001938000F033711000CB
:102F1000930300006318710493019001B700FF0050
:102F20009B80F00F33F1000093030000631C7102DB
:102F30009301A001B370000093030000639470023A
:102F40009301B001B71011119B801011372122227B
:102F50001B01212233F02000930300006314700052
:102F6000631A300013951100630005001365150006
:102F7000730000001305100073000000731000C000
:082F8000010101010101010141
:102F8800417373657274696F6E206661696C6564FC
:102F98003A2061646472203E3D202831554C203C23
:102FA8003C203132292026262061646472203C208E
:102FB8003633202A202831554C203C3C20313229F8
:102FC8000A00000000000000417373657274696FA5
:102FD8006E206661696C65643A20212870745B33E1
:102FE8005D5B616464722F2831554C203C3C203174
:102FF80032295D20262030783038302920262620B6
:103008006361757365203D3D203078660A000000D5
:10301800417373657274696F6E206661696C65646B
:103028003A206E6F64650A00417373657274696F44
:103038006E206661696C65643A20757365725F6DB0
:10304800617070696E675B616464722F2831554CDA
:10305800203C3C203132295D2E61646472203D3D64
:1030680020300A0000000000417373657274696FB4
:103078006E206661696C65643A202122696C6C6512
:1030880067616C20696E737472756374696F6E2200
:103098000A00000000000000417373657274696FD4
:1030A8006E206661696C65643A2070745B335D5BA1
:1030B800616464722F2831554C203C3C2031322900
:1030C8005D20262030783034300A000000000000EF
:1030D800417373657274696F6E206661696C6564AB
:1030E8003A2070745B335D5B616464722F283155DC
:1030F8004C203C3C203132295D2026203078303865
:10310800300A000000000000417373657274696F33
:103118006E206661696C65643A2074662D3E657040
:103128006320252034203D3D20300A0000000000A7
:10313800417373657274696F6E206661696C65644A
:103148003A202122756E6578706563746564206520
:103158007863657074696F6E220A000000000000D1
:10316800417373657274696F6E206661696C65641A
:103178003A202122756E737570706F7274656420C1
:0C31880073617470206D6F6465220A0092
:040000058000000077
:00000001FF
